:020000040000FA
:0400000075EF0BF09D
:08000800026ED8CF01F0E0CF39
:1000100000F0F2A419EF00F081721A2E14EF00F034
:10002000D59E038019EF00F0670ED76E690ED66E6D
:10003000F29400C0E0FF025001C0D8FF10000A0E89
:10004000286E2650296E27502A6E261E271E272A24
:10005000D8B4262AF80E256E0000252E2CEF00F0CD
:1000600000000000272AD8B4263E2AEF00F02950CD
:10007000266E2A50276E282E25EF00F0120083905E
:10008000839283945BEF00F08380839283945BEF91
:1000900000F08390838283945BEF00F083808382FF
:1000A00083945BEF00F08390839283845BEF00F096
:1000B000838083928384829A828A1200238E76EFD1
:1000C00000F0238C76EF00F0238A76EF00F023888F
:1000D00076EF00F0239E76EF00F0239C76EF00F0A1
:1000E000239A76EF00F0239876EF00F058EC00F0BA
:1000F00023C083FF3FEF00F0030E8D6E8B90000E48
:100100002D6E000E2B6E12000652D8B405060606A0
:1001100005C08CFF8B808B9006C08CFF8D848D94E6
:100120002FC083FF8D928D820652D8B40506060635
:1001300005C08CFF8B808B9006C08CFF8D848D94C6
:1001400030C083FF8D928D82120005C08CFF8B80A2
:100150008B9006C08CFF8D848D94FF0E956E836A04
:100160008D9083CF30F08D80956A062AD8B4052A09
:1001700005C08CFF8B808B9006C08CFF8D848D9486
:10018000FF0E956E836A8D9083CF2FF08D80956AD8
:10019000062AD8B4052A12000852D8B40706080661
:1001A00007C08CFF8B808B9008C08CFF8D848D9452
:1001B0002FC083FF8D928D820852D8B4070608069F
:1001C00007C08CFF8B808B9008C08CFF8D848D9432
:1001D00030C083FF8D928D82120007C08CFF8B8010
:1001E0008B9008C08CFF8D848D94FF0E956E836A72
:1001F0008D9083CF30F08D80956A082AD8B4072A75
:1002000007C08CFF8B808B9008C08CFF8D848D94F1
:10021000FF0E956E836A8D9083CF2FF08D80956A47
:10022000082AD8B4072A12002BC08CFF8B808B9031
:100230002DC08CFF8D848D9430C083FF8D928D8274
:100240002D2AD8B42B2A2BC08CFF8B808B902DC0ED
:100250008CFF8D848D942FC083FF8D928D82120030
:100260002BC08CFF8B808B902DC08CFF8D848D9448
:1002700030C083FF8D928D8212002BC08CFF8B804B
:100280008B902DC08CFF8D848D94FF0E956E836AAC
:100290008D9083CF30F08D80956A2D2AD8B42B2A8B
:1002A0002BC08CFF8B808B902DC08CFF8D848D9408
:1002B000FF0E956E836A8D9083CF2FF08D80956AA7
:1002C00012002BC08CFF8B808B902DC08CFF8D84F7
:1002D0008D94FF0E956E836A8D9083CF30F08D8064
:1002E000956A1200166A306A2F6A03920F0E16146E
:1002F000D8A47FEF01F0A5EC01F084EF01F0070E28
:100300001614D8B49EEC01F061EC01F0305014ECFE
:100310000FF0200E27EC02F0200E305CD8B093EFE7
:1003200001F02E0E306E30C0EEFF2D2AD8B42B2AED
:10033000162AD8B4B6EF01F076EF01F02D0E27ECB7
:1003400002F0200E27EC02F0120003B2B6EC01F02E
:1003500003822CEC02F03CEC0FF03A0E27EC02F09A
:10036000200E27EC02F001EE00F01200200E27EC28
:1003700002F0200E27EC02F001EE00F0EE5027EC28
:1003800002F0E9A8BEEF01F01200306E2F6A000EF5
:100390002D6E000E2B6E30EC01F02D2AD8B42B2AD6
:1003A000D8B41200CBEF01F0306A2F6A000E2D6E28
:1003B000000E2B6E2BC030F030EC01F02D2AD8B49B
:1003C0002B2AD8B41200DAEF01F02F6E306A000E3B
:1003D0002D6E000E2B6E039261EC01F02F50305CFD
:1003E000D8A4FBEF01F02D2AD8B42B2AD8B41CEFE7
:1003F00002F0ECEF01F00382000EF86E220EF76EB1
:10040000400EF66EF7EC0EF03CEC0FF0200E27ECF1
:1004100002F027EC02F02F5014EC0FF0000EF86EF3
:10042000220EF76E6A0EF66EF7EC0EF0305014ECFA
:100430000FF02CEC02F0120003B21200000EF86E66
:10044000220EF76E500EF66EF7EC0EF01200ACA214
:1004500027EF02F0AD6E12000D0E27EC02F00A0E2F
:1004600027EC02F012003E0E27EC02F0200E27ECE3
:1004700002F01200ABB23FEF02F0AE5012005F0E7E
:1004800027EC02F0580E27EC02F05F0E27EC02F08A
:10049000AB98AB8812000450CCEC0EF0829203B003
:1004A0005FEF02F09EAA4FEF02F08282D5EC0EF0D1
:1004B000AE50ABA21200AB98AB880380000C8282D6
:1004C000D5EC0EF0000C7AEC02F086EC02F0A0EC19
:1004D00002F0376A386A000EACEC02F08EEC02F0E3
:1004E000326A336A346A356A000EC8EC02F07EEC78
:1004F00002F012003C94F80EE4EF02F03C84C00ECF
:10050000E4EF02F0A00E3C92E4EF02F0B00E3C8269
:10051000E4EF02F03CA097EF02F000003C903CA218
:1005200095EF02F0500EE4EF02F0839412003C804D
:100530003CA29EEF02F0580EE4EF02F0838412001A
:10054000400EE4EF02F0420EE4EF02F0440EE4EF5E
:1005500002F0460EE4EF02F0396E18093A6E385098
:100560003B6EE6EC02F0395009093A6E37503B6EAB
:10057000E6EF02F03CA0C3EF02F00000000EC8EC72
:1005800002F08EEF02F0040EC8EC02F097EF02F0DA
:10059000366E30093A6E35503B6EE6EC02F036505E
:1005A00021093A6E34503B6EE6EC02F036503209C7
:1005B0003A6E33503B6EE6EC02F0365023093A6E49
:1005C00032503B6EE6EF02F03A6E3B6A53EC00F0BD
:1005D000100E3D6E3AAE83923ABE83828380839042
:1005E0003B363A363D2EEAEF02F03FEC00F01200C7
:1005F00063EC02F07EEC02F02C0E3E6E82EC03F017
:1006000005EC03F07AEC02F01200FF0E406E71EC84
:1006100003F0010E416E000E326E030E336E030EB8
:10062000346EC00E356EBAEC02F03CA00BEF03F056
:10063000000E266E490E276E1FEC00F0000E326E83
:10064000010E336EF70E346E510E356EBAEC02F0B9
:10065000000E266E490E276E1FEC00F0412E0BEFA8
:1006600003F0000E266E010E276E1FEC00F0040E44
:10067000416E97EC02F0000E266E120E276E1FECF4
:1006800000F08EEC02F0000E266E120E276E1FECAC
:1006900000F0412E39EF03F0000E266E020E276E99
:1006A0001FEC00F0020E416E97EC02F0000E266E79
:1006B000240E276E1FEC00F08EEC02F0000E266E6A
:1006C000240E276E1FEC00F0412E54EF03F0402E55
:1006D00007EF03F0000E266E020E276E1FEC00F0EF
:1006E0001200000E326E010E336E920E346EA70EA3
:1006F000356EBAEC02F0000E266E050E276E1FEC6A
:1007000000F01200000E326E020E336E7D0E346E5B
:10071000880E356EBAEC02F0010E266E2C0E276E96
:100720001FEC00F0000E326E010E336E920E346E2E
:10073000A70E356EBAEC02F0000E266E0A0E276E7A
:100740001FEC00F08AEC02F0010E266E2C0E276ED4
:100750001FEC00F08AEC02F0000E266E1E0E276ED3
:100760001FEC00F03F6A3C8E070E406E3E32D8A070
:10077000C7EF03F03F2A000E326E010E336E710E8A
:10078000346E190E356EBAEC02F0D1EF03F0000EA4
:10079000326E010E336EB40E346E350E356EBAEC19
:1007A00002F0000E266E1E0E276E1FEC00F0402E8B
:1007B000B6EF03F03CAEE5EF03F03C9E402A3FA0CD
:1007C000C7EF03F03FB0BAEF03F0000E326E010E38
:1007D000336E920E346EA70E356EBAEC02F0000E38
:1007E000266E1E0E276E1FEC00F0120049EC00F082
:1007F000836A300E426E3EEC04F03EEC04F03EECB8
:1008000004F0200E426E3EEC04F0280E31EC04F0B1
:100810000C0E31EC04F028EC04F0060E31EC04F080
:100820003FEC00F012000C0E31EF04F0080E31EF37
:1008300004F00F0E31EF04F00E0E31EF04F00C0E49
:1008400031EF04F0100E31EF04F0140E31EF04F02C
:10085000010E31EF04F0426E800E421031EF04F0D1
:10086000020E839435EF04F083848396426E3EEC4F
:1008700004F0423A3EEC04F042381200000E266EBC
:10088000060E276E1FEC00F00F0E8316F00E4214BA
:100890008312838083901200516A446A456A466AD3
:1008A000476A486A496A4A6A4B6A180E4F6E4C3664
:1008B0004D364E3600EE44F0080E506EEF360A0EFE
:1008C000EF5CD8B0EF6EEE52502E5EEF04F04F2E7C
:1008D00057EF04F01200516A446A456A466A476A53
:1008E000486A496A4A6A4B6A4C500F0B446E4C384E
:1008F0000F0B456E4D500F0B466E4D380F0B476E6C
:100900004E500F0B486E4E380F0B496E1200516A55
:10091000456E45380F0BF60FD8B0070F3A0F451A42
:100920004518451A0F0BF60FD8B0070F3A0F446E53
:100930001200516A4F6A00EE44F04C32D8A0000E0B
:10094000D8B0010EEF6EEE524F2A4FA69DEF04F085
:100950001200506E070E5016D8A4B1EF04F0080E26
:10096000506E00EE44F05152D8B4BBEF04F0EE529A
:10097000512EB7EF04F05004EB50300F27EC02F08B
:10098000502EBBEF04F0120003940A0E046E4BECE1
:1009900002F003B0020C3A0EAE5CD8A4C4EF04F02F
:1009A000818829EC05F003B0020C526E576E29ECD9
:1009B00005F003B0020C536E572629EC05F003B086
:1009C000020C546E572629EC05F003B0020C556E4C
:1009D00057265552D8A41DEF05F05252D8B410EF47
:1009E00005F029EC05F003B0020C566E572653C0F3
:1009F0008CFF8B808B9054C08CFF8D848D9456C05F
:100A000083FF8D928D82542AD8B4532A5452D8A48D
:100A10000DEF05F02E0E27EC02F05206EDEF04F07C
:100A200029EC05F003B0020C5724D8A4010C54C0E3
:100A30002DF053C02BF0C4EF04F05504D8A4C4EF3C
:100A400004F029EC05F003B0020C5724D8A4010CE3
:100A5000000C4BEC02F003A443EF05F00396146E78
:100A60001B0E145CD8B4038003B01200145027ECA2
:100A700002F0200E145CD8B40380D8B4038614505E
:100A800003B627EC02F003B0120066EC05F0136E1B
:100A9000133A4BEC02F003A45FEF05F0146E1B0E4B
:100AA000145CD8B4038003B01200145027EC02F099
:100AB000200E145CD8B40380D8B40386145003B05D
:100AC000120066EC05F0131213501200146E300E73
:100AD000145EF00E1414D8B470EF05F0070E145E17
:100AE00014501200190EC86E080EC66EC68A120087
:100AF0009E96C58091EF05F0C58891EF05F078ECE2
:100B000005F013508AEC05F090EC05F0C5AC12002E
:100B10007FEF05F0C96E91EF05F0C58691EF05F006
:100B2000C5849EA691EF05F09E96120078EC05F024
:100B3000300E8AEC05F0F7EF0BF0596A300E5910C1
:100B40008AEC05F0F7EF0BF090EC05F0F7EF0BF007
:100B50002CEC02F0530E27EC02F03D0E27EC02F0D5
:100B600078EC05F0310E8AEC05F08DEC05F0C9CF7C
:100B70005BF090EC05F05B500BEC0FF02CEC02F00E
:100B8000F7EF0BF01E0E046E2CEC02F0000EF86E68
:100B9000230EF76ECE0EF66EF7EC0EF00384010E08
:100BA00049EC0BF003B081EF06F04CC059F02CEC8F
:100BB00002F0070E5916000EF86E230EF76EEA0EBD
:100BC000F66EF7EC0EF085EC06F0B4EC06F0E3EC14
:100BD00006F011EC07F0500E27EC02F03D0E27EC6A
:100BE00002F05B500BEC0FF0200E27EC02F0200E11
:100BF00027EC02F0540E27EC02F03D0E27EC02F039
:100C00005C500BEC0FF0200E27EC02F0200E27ECCE
:100C100002F0430E27EC02F03D0E27EC02F05A5092
:100C200021EC0FF0200E27EC02F0200E27EC02F052
:100C30004F0E27EC02F03D0E27EC02F05D5021EC48
:100C40000FF00D0E27EC02F082929EAA25EF06F01F
:100C500082823AEC02F0116E1B0E115CD8B481EF67
:100C600006F02B0E115CD8B4C9EF08F02D0E115C04
:100C7000D8B4D0EF08F02A0E115CD8B4CCEF08F04D
:100C80005F0E115CD8B4D3EF08F02E0E115CD8B40F
:100C9000D7EF08F02C0E115CD8B4DEEF08F03A0E56
:100CA000115CD8B4DAEF08F03B0E115CD8B4E1EF78
:100CB00008F0530E115CD8B483EF07F0540E115CAA
:100CC000D8B49BEF07F0430E115CD8B4B3EF07F034
:100CD000580E115CD8B41AEF08F0780E115CD8B435
:100CE00032EF08F0450E115CD8B44AEF08F04F0E11
:100CF000115CD8B462EF08F0070E27EC02F0EBEFBE
:100D000005F02CEC02F0F7EF0BF078EC05F0300E6C
:100D10008AEC05F0000E266E020E276E1FEC00F026
:100D2000300E59108AEC05F0000E266E020E276E6A
:100D30001FEC00F090EC05F078EC05F0310E8AEC39
:100D400005F0000E266E020E276E1FEC00F08DECF3
:100D500005F0000E266E020E276E1FEC00F0C9CFC4
:100D60005BF090EC05F0120078EC05F0300E8AECA8
:100D700005F0000E266E020E276E1FEC00F0380EF6
:100D800059108AEC05F0000E266E020E276E1FEC3D
:100D900000F090EC05F078EC05F0310E8AEC05F0EF
:100DA000000E266E020E276E1FEC00F08DEC05F093
:100DB000000E266E020E276E1FEC00F0C9CF5CF00D
:100DC00090EC05F0120078EC05F0300E8AEC05F09E
:100DD000000E266E020E276E1FEC00F0480E8AEC05
:100DE00005F0000E266E020E276E1FEC00F090EC50
:100DF00005F078EC05F0310E8AEC05F0000E266E59
:100E0000020E276E1FEC00F08DEC05F0000E266E32
:100E1000020E276E1FEC00F0C9CF5AF090EC05F0DF
:100E2000120078EC05F0300E8AEC05F0000E266E0C
:100E3000020E276E1FEC00F0600E8AEC05F0000E2B
:100E4000266E020E276E1FEC00F090EC05F078EC99
:100E500005F0310E8AEC05F0000E266E020E276EAC
:100E60001FEC00F08DEC05F0000E266E020E276ED2
:100E70001FEC00F0C9CF5DF090EC05F0120078ECAB
:100E800005F0300E8AEC05F0000E266E020E276E7D
:100E90001FEC00F0000E59108AEC05F0000E266ED3
:100EA000020E276E1FEC00F05B508AEC05F0000E7E
:100EB000266E020E276E1FEC00F090EC05F0EBEFB3
:100EC00005F078EC05F0300E8AEC05F0000E266E89
:100ED000020E276E1FEC00F0080E59108AEC05F088
:100EE000000E266E020E276E1FEC00F05C508AEC9E
:100EF00005F0000E266E020E276E1FEC00F090EC3F
:100F000005F0EBEF05F078EC05F0300E8AEC05F01B
:100F1000000E266E020E276E1FEC00F0100E8AECFB
:100F200005F0000E266E020E276E1FEC00F090EC0E
:100F300005F0EBEF05F078EC05F0300E8AEC05F0EB
:100F4000000E266E020E276E1FEC00F0180E8AECC3
:100F500005F0000E266E020E276E1FEC00F090ECDE
:100F600005F0EBEF05F01E0E046E000EF86E250E78
:100F7000F76E320EF66EF7EC0EF0000EF86E250EE0
:100F8000F76E320EF66EF7EC0EF00D0E27EC02F057
:100F9000000EF86E240EF76EF60EF66EF7EC0EF0FD
:100FA0005A5021EC0FF0000EF86E250EF76E2E0E43
:100FB000F66EF7EC0EF003841AEC0BF003B002EFC0
:100FC00008F013C05AF078EC05F0300E8AEC05F00A
:100FD000000E266E020E276E1FEC00F0400E8AEC0B
:100FE00005F0000E266E020E276E1FEC00F05A5020
:100FF0008AEC05F0000E266E020E276E1FEC00F044
:1010000090EC05F00D0E27EC02F0000EF86E250EA8
:10101000F76E320EF66EF7EC0EF0000EF86E250E3F
:10102000F76E320EF66EF7EC0EF00D0E27EC02F0B6
:10103000EBEF05F078EC05F0300E8AEC05F0000ED1
:10104000266E020E276E1FEC00F0500E8AEC05F0A3
:10105000000E266E020E276E1FEC00F090EC05F0DD
:10106000E3EF05F078EC05F0300E8AEC05F0000EA9
:10107000266E020E276E1FEC00F0580E8AEC05F06B
:10108000000E266E020E276E1FEC00F090EC05F0AD
:10109000E3EF05F078EC05F0300E8AEC05F0000E79
:1010A000266E020E276E1FEC00F0280E8AEC05F06B
:1010B000000E266E020E276E1FEC00F090EC05F07D
:1010C000E3EF05F01E0E046E000EF86E250EF76EAF
:1010D000320EF66EF7EC0EF0000EF86E250EF76E7F
:1010E000320EF66EF7EC0EF00D0E27EC02F0000E4D
:1010F000F86E250EF76E100EF66EF7EC0EF05D50E2
:1011000021EC0FF0000EF86E250EF76E2E0EF66E27
:10111000F7EC0EF003841AEC0BF003B0B1EF08F01B
:1011200013C05DF078EC05F0300E8AEC05F0000E8F
:10113000266E020E276E1FEC00F0680E8AEC05F09A
:10114000000E266E020E276E1FEC00F05D508AEC3A
:1011500005F0000E266E020E276E1FEC00F090ECDC
:1011600005F00D0E27EC02F0000EF86E250EF76E5E
:10117000320EF66EF7EC0EF0000EF86E250EF76EDE
:10118000320EF66EF7EC0EF00D0E27EC02F0E3EFE8
:1011900005F05B2A3FEF07F00A0E5B263FEF07F0F2
:1011A0005B063FEF07F00A0E5B5E3FEF07F05C2A3D
:1011B00061EF07F00A0E5C2661EF07F05C0661EF55
:1011C00007F00A0E5C5E61EF07F00BEC09F003B06C
:1011D000F6EF08F02CEC02F0000EF86E230EF76E1E
:1011E000220EF66EF7EC0EF06EEC09F0F7EF0BF056
:1011F0000BEC09F003B009EF09F02CEC02F0000E43
:10120000F86E230EF76E220EF66EF7EC0EF036EC4B
:1012100009F0F7EF0BF02CEC02F0000EF86E210E47
:10122000F76ED80EF66EF7EC0EF01E0E046E038409
:1012300029EC05F003B035EF09F01352D8B42BEFC9
:1012400009F01306D8B42FEF09F01306D8B433EF22
:1012500009F0E5EF08F0A00E586E35EF09F0A20E88
:10126000586E35EF09F0A40E586E12000392166AFC
:10127000306A2F6A000E2D6E000E2B6E78EC05F092
:1012800058502BBEE886E8CF13F08AEC05F02B50BF
:101290008AEC05F02D508AEC05F061EC01F030503D
:1012A0008AEC05F02D2AD8B42B2AD8B4038203B2D5
:1012B00060EF09F0162A16BC60EF09F04DEF09F057
:1012C00090EC05F02E0E27EC02F07FEC05F0166A8C
:1012D00003A23EEF09F02CEC02F012000392166A12
:1012E000306A2F6A000E2D6E000E2B6E78EC05F022
:1012F00058502BBEE8868AEC05F02B508AEC05F09E
:101300002D508AEC05F090EC05F078EC05F0585083
:10131000E8802BBEE8868AEC05F08DEC05F0C9CF9D
:1013200030F030EC01F02D2AD8B42B2AD8B4B0EF2D
:1013300009F0162A16ACA1EF09F02E0E27EC02F0E8
:10134000166A03B2ACEF09F02BAEACEF09F00382E2
:1013500090EC05F076EF09F07CEC05F08DEF09F0EC
:1013600090EC05F02CEC02F01200900E586E2CEC74
:1013700002F0000EF86E230EF76E4E0EF66EF7ECCE
:101380000EF0D0EC09F030500BEC0FF0200E27ECF3
:1013900002F0430E27EC02F02CEC02F0F7EF0BF01A
:1013A00078EC05F058508AEC05F0000E8AEC05F058
:1013B00090EC05F078EC05F05850E8808AEC05F0E8
:1013C0008DEC05F0C9CF30F090EC05F01200D00E96
:1013D000586E2CEC02F0000EF86E230EF76E620EC3
:1013E000F66EF7EC0EF0000EF86E230EF76E9A0E06
:1013F000F66EF7EC0EF0000EF86E230EF76EB60EDA
:10140000F66EF7EC0EF04EEC0AF085EC0AF0200ECA
:1014100027EC02F0200E27EC02F0A3EC0AF02CECF3
:1014200002F0000EF86E230EF76EB60EF66EF7ECB5
:101430000EF0C1EC0AF02CEC02F0F7EF0BF078ECB8
:1014400005F058508AEC05F0000E8AEC05F090EC9F
:1014500005F078EC05F05850E8808AEC05F08DEC4A
:1014600005F0C9CF30F090EC05F0309E78EC05F037
:1014700058508AEC05F0000E8AEC05F030508AECEA
:1014800005F090EC05F012001B6A1C6A1D6A1E6ACA
:101490001F6A206A216A70EC0AF0120000EE1BF04D
:1014A00078EC05F058508AEC05F0000E8AEC05F057
:1014B00090EC05F078EC05F05850E8808AEC05F0E7
:1014C000070E506E8DEC05F0C9CFEEFF502E6CEF7D
:1014D0000AF090EC05F012007CEC05F062EF0AF0E7
:1014E00000EE1BF078EC05F058508AEC05F0000E89
:1014F0008AEC05F0070E506EEE508AEC05F0502E87
:101500007CEF0AF090EC05F012001FC04EF020C0F6
:101510004DF021C04CF06BEC04F0040E516E020E45
:10152000A9EC04F02E0E27EC02F0020E516E020E12
:10153000A9EC04F02E0E27EC02F0000E516E020E04
:10154000A9EC04F012001DC04EF01CC04DF01BC0F1
:101550004CF06BEC04F0040E516E020EA9EC04F09A
:101560003A0E27EC02F0020E516E020EA9EC04F0C6
:101570003A0E27EC02F0000E516E020EA9EC04F0B8
:1015800012001E0E046E0384020E49EC0BF003B031
:1015900019EF0BF04D384C124CC01FF02E0E27ECFB
:1015A00002F00384020E49EC0BF003B019EF0BF0CC
:1015B0004D384C124CC020F02E0E27EC02F0038464
:1015C000020E49EC0BF003B019EF0BF04D384C1242
:1015D0004CC021F0200E27EC02F0200E27EC02F088
:1015E0000384020E49EC0BF003B019EF0BF04D38F9
:1015F0004C124CC01DF03A0E27EC02F00384020E90
:1016000049EC0BF003B019EF0BF04D384C124CC005
:101610001CF03A0E27EC02F00384020E49EC0BF0AA
:1016200003B019EF0BF04D384C124CC01BF070ECAE
:101630000AF01200136A080E506E4BEC02F0146EA2
:1016400003A429EF0BF01B0E145CD8B4038003B085
:10165000120003B01200300E145CD8B43DEF0BF052
:10166000310E145CD8B440EF0BF003A41DEF0BF067
:10167000070E27EC02F01DEF0BF0D89041EF0BF0B6
:10168000D8801336145027EC02F0502E1DEF0BF0CB
:1016900012004C6A4D6A4E6A00EE4CF0506E030E1A
:1016A0005016D8A456EF0BF0030E506E4BEC02F020
:1016B000146E03A465EF0BF01B0E145CD8B403800A
:1016C00003B01200145027EC02F003B0120070ECCB
:1016D0000BF0500414C0EBFF502E56EF0BF012002D
:1016E000300E145E0F0E141412008198116A136AE2
:1016F000132E78EF0BF0112E77EF0BF0D0A289EFBD
:101700000BF08188D0A087EF0BF0B8EF0BF0B8EFAB
:101710000BF00001030E926E040E936EDC0E946EBD
:10172000000E956E000E966E000ED06E000EF26EDC
:10173000C00EF16E000EF06E000E9F6E200E9D6EBC
:10174000000EA26E000EA06E000EA56E000EA36E1F
:10175000200EAC6E900EAB6E400EAF6E070EB46EE8
:10176000000EB56E070ED56E810EC26ECE0EC16E26
:101770003FEC00F07CEC00F063EC02F072EC05F062
:10178000F6EC03F0136A81928198F28EF28A039448
:10179000800E226E236A76EC00F02CEC02F02A0E0A
:1017A00027EC02F0050ECCEC0EF0829203B0EAEFCB
:1017B0000BF09EAAD6EF0BF082823AEC02F0116E8B
:1017C0002D0E115CD8A4EAEF0BF08282D5EC0EF05E
:1017D000EFEF0BF08282D5EC0EF000EF18F0000E68
:1017E000F86E200EF76E4E0EF66EF7EC0EF033EC40
:1017F00002F082929EAAFAEF0BF082823AEC02F09B
:10180000116E27EC02F0200E27EC02F03F0E115C67
:10181000D8B42AEF0FF03E0E115CD8B48BEF0DF068
:101820003C0E115CD8B4C4EF0DF0230E115CD8B49B
:101830002BEF0EF02F0E115CD8B457EF0EF05C0EAC
:10184000115CD8B4F3EF0DF03D0E115CD8B46EEF1F
:101850000EF05F0E115CD8B476EF0EF02A0E115C1C
:10186000D8B400EF18F0260E115CD8B4F8EF08F0E9
:10187000250E115CD8B4E5EF08F0400E115CD8B429
:1018800090EF0CF0210E115CD8B4B5EF09F07E0E8C
:10189000115CD8B4E7EF09F02D0E115CD8B4C2EF9B
:1018A00005F02B0E115CD8B4CFEF0CF0A70E115C35
:1018B000D8B456EF0DF0300E115CD8B47CEF0DF0BB
:1018C000310E115CD8B478EF0DF0320E115CD8B443
:1018D000EEEF0CF0330E115CD8B4F3EF0CF0340ED5
:1018E000115CD8B4F8EF0CF07C0E115CD8B449EF61
:1018F0000DF011C012F02BC08CFF8B808B902DC08F
:101900008CFF8D848D9411C083FF8D928D822D2A42
:10191000D8B42B2A3CEC0FF02CEC02F0F7EF0BF0D4
:101920003CEC0FF02CEC02F0156A166A2D50165C98
:10193000D8A4A4EF0CF02B50155CD8A4A4EF0CF0A5
:101940002CEC02F0F7EF0BF015C08CFF8B808B9026
:1019500016C08CFF8D848D94FF0E956E836A8D90DA
:1019600083CF11F08D80956A115027EC02F0162A72
:10197000D8B4152A96EF0CF0A5EC00F0305027EC07
:1019800002F02F5027EC02F02CEC02F0F7EF0BF0F6
:101990002F6A12C030F084EC00F0F7EF0BF049EC46
:1019A00000F028EC04F00388000EF86E250EF76EA8
:1019B000840EF66EF7EC0EF0039849EC00F0400E42
:1019C0002BEC04F00388000EF86E250EF76E8A0EDD
:1019D000F66EF7EC0EF00398F7EF0BF049EC00F021
:1019E0008380F7EF0BF083903FEC00F0F7EF0BF004
:1019F000F6EC03F0F7EF0BF053EC00F07EEC02F0A6
:101A0000000E326E010E336EF70E346E510E356ECF
:101A1000BAEC02F03FEC00F0F7EF0BF053EC00F003
:101A20007AEC02F03FEC00F0F7EF0BF02CEC02F058
:101A3000000EF86E250EF76E5A0EF66EF7EC0EF0ED
:101A4000F8EC02F0F7EF0BF0C46AC36AC284C2B4C8
:101A500027EF0DF04E6AC4CF4DF0C3CF4CF04CECE5
:101A600004F0040EA9EC04F0200E27EC02F080A292
:101A70002D0E80B22B0E27EC02F0200E27EC02F088
:101A8000D0EC09F030500BEC0FF02CEC02F0F7EF3B
:101A90000BF02CEC02F04F0E27EC02F04B0E27EC73
:101AA00002F0200E27EC02F024EF0DF02CEC02F0F7
:101AB000000EF86E220EF76E860EF66EF7EC0EF044
:101AC0001E0E046E038429EC05F003B0F7EF0BF053
:101AD000200E27EC02F0135021EC0FF058EC00F030
:101AE00013C083FF3FEC00F02CEC02F0F7EF0BF09B
:101AF00067EC00F0F7EF0BF073EC00F0F7EF0BF092
:101B0000C46AC36AC284C2B483EF0DF01200D884E1
:101B100080A2D89412002CEC02F0000EF86E210E78
:101B2000F76EF40EF66EF7EC0EF0000EF86E220E65
:101B3000F76E120EF66EF7EC0EF0200E27EC02F0A8
:101B40000A0E0BEC0FF0200E27EC02F0000EF86EE0
:101B5000220EF76E1A0EF66EF7EC0EF02CEC02F079
:101B6000C4EC04F0136E2CEC02F0000EF86E210EA3
:101B7000F76ECA0EF66EF7EC0EF013500BEC0FF08A
:101B80002CEC02F0F7EF0BF02BC02CF02DC02EF058
:101B90002CEC02F0000EF86E220EF76EAC0EF66E14
:101BA000F7EC0EF01E0E046E038429EC05F003B072
:101BB000EFEF0DF013C02BF03A0E27EC02F0038488
:101BC00029EC05F003B0EFEF0DF013C02DF02CEC75
:101BD00002F072EC01F02CC02BF02EC02DF02CEC9A
:101BE00002F0F7EF0BF02BC02CF02DC02EF02CECF8
:101BF00002F0000EF86E220EF76EAC0EF66EF7ECE9
:101C00000EF01E0E046E038429EC05F003B027EFDE
:101C10000EF013C02BF03A0E27EC02F0038429ECEF
:101C200005F003B027EF0EF013C02DF0000EF86E94
:101C3000220EF76E700EF66EF7EC0EF061EC01F00E
:101C4000305014EC0FF02CC02BF02EC02DF02CECEB
:101C500002F0F7EF0BF02BC02CF02DC02EF02CEC87
:101C600002F0000EF86E220EF76E860EF66EF7EC9E
:101C70000EF01E0E046E038429EC05F02CEC02F02D
:101C800003B0F7EF0BF0000EF86E220EF76E220E87
:101C9000F66EF7EC0EF01350C5EC01F01350E5ECC6
:101CA00001F02CC02BF02EC02DF0F7EF0BF02BC065
:101CB0002CF02DC02EF02CEC02F0E86AC5EC01F0FF
:101CC000000EF86E220EF76E5A0EF66EF7EC0EF05E
:101CD0002CC02BF02EC02DF0F7EF0BF02CEC02F007
:101CE0003CEC0FF02CEC02F0F7EF0BF02CEC02F0D8
:101CF000000EF86E220EF76EC40EF66EF7EC0EF0C4
:101D00001E0E046E038429EC05F003B0C8EF0EF03C
:101D100013C02BF03A0E27EC02F0038429EC05F0F7
:101D200003B0C8EF0EF013C02DF02CEC02F0000E43
:101D3000F86E220EF76EE60EF66EF7EC0EF02CEC57
:101D400002F03CEC0FF03A0E27EC02F0166A200E7F
:101D500027EC02F061EC01F0305014EC0FF02D0E86
:101D600027EC02F0038429EC05F003B6BFEF0EF078
:101D700003B0C8EF0EF013C083FF8D928D822D2A21
:101D8000D8B42B2A162A16A6A7EF0EF09FEF0EF056
:101D90002CEC02F0F7EF0BF01A6E670ED76E690E9F
:101DA000D66EF2940390D58E1200D59E1200176A5B
:101DB000186A196ED8901936183619361836000E6A
:101DC0001924F66E200E1820F76E000E1720F86EFC
:101DD0000900F5CF17F00900F5CF18F00900F5CF8D
:101DE00019F017C0F8FF18C0F7FF19C0F6FF03B8C5
:101DF00049EC00F00900F550D8B407EF0FF003A844
:101E000027EC02F003B834EC04F0FAEF0EF003B85C
:101E10003FEC00F012004E6A4D6A4C6E4CEC04F040
:101E2000030EA9EC04F01200456A446A87EC04F042
:101E300045C0E8FF27EC02F044C0E8FF27EC02F0C1
:101E400012004E6A4D6A4C6E99EC04F0080EA9EC33
:101E500004F01200000EF86E200EF76E4E0EF66EB5
:101E6000F7EC0EF0000EF86E200EF76E660EF66EB2
:101E7000F7EC0EF0F7EF0BF02B5014EC0FF02D50A9
:061E800014EC0FF012004B
:102000000020220000202E0000204E00002066004C
:102010000021CA000021F4000022120000221A0050
:102020000000537472696E6720310D0A000053740A
:1020300072696E6720320D0A00000D0A57656C63E5
:102040006F6D6520746F204950530D0A00000D0A12
:10205000495053204D6F6E69746F722056312E3087
:102060000D0A0D0A00003F202053686F7720746826
:1020700069732068656C702073637265656E0D0A04
:102080003E20204C6F616420496E74656C20484589
:10209000582046696C6520200D0A3C202044756D4F
:1020A00070205352414D20746F20436F6E736F6CDC
:1020B00065200D0A23202054657374205352414D2E
:1020C0002020202020202020202020200D0A2F202A
:1020D00020436C656172205352414D202020202006
:1020E0002020202020200D0A5C202053686F7720BC
:1020F0004279746520617420416464726573732051
:102100000D0A3D202053686F772041646472657327
:102110007320506F696E746572200D0A5F20205322
:102120006574204164647265737320506F696E74C6
:10213000657220616E642065646974205352414D5C
:102140000D0A26202053617665205352414D202DE3
:102150002D3E20454550524F4D200D0A252020523E
:102160006573746F726520454550524F4D202D2D7B
:102170003E205352414D0D0A7E202053686F772F29
:10218000536574207265616C2074696D6520636CA1
:102190006F636B200D0A2D2020436F6E6669677593
:1021A000726520536572766F73200D0A2A202052C3
:1021B0006573746172742053797374656D20202087
:1021C000202020200D0A0D0A00005254433A20001E
:1021D0004F4B00004552520053656C6563742052AA
:1021E000414D2062616E6B202830302C30312C3014
:1021F00032293A00537461727420494E54454C2080
:102200004845582066696C652075706C6F61640D77
:102210000A0054696D656F7574007365636F6E6451
:102220007300436865636B696E67205352414D20AC
:102230002D20706C6561736520776169740D0A00EB
:102240005352414D204572726F722061743A2000E2
:102250005352414D204F4B0D0A005352414D2043E4
:102260006C65617265640D0A0000203C3E20000030
:10227000203D2000456E7465722048455820566107
:102280006C75653A2000456E74657220484558208B
:1022900056616C756520283220436861727329206D
:1022A000746F2077726974653A200000456E74651A
:1022B000722041646472657373202848483A4C4C1C
:1022C000293A200053657420416464726573732059
:1022D000506F696E74657220746F202848483A4CBC
:1022E0004C293A20000028455343293D43616E6341
:1022F000656C2C20285350414345293D536B697030
:102300002C203220415343494920486578204368B6
:10231000617273206368616E6765732076616C75A6
:1023200065004F6E6520222E22203D20363420424B
:10233000797465730D0A00004F6E6520222E2220ED
:102340003D203235362042797465730D0A00426FA4
:102350006172642074656D70657261747572653A3E
:10236000200053686F772F53657420436C6F636B45
:102370002C2028455343293D43616E63656C2C2016
:102380003220446967697473206368616E6765739E
:102390002076616C75650D0A0000436C6F636B3AC3
:1023A0002044442E4D4D2E5959202048483A4D4D39
:1023B0003A53530D0A0020202020202020004932CB
:1023C0004320536572766F746573740D0A00456E11
:1023D00074657220536572766F206E756D626572DA
:1023E0002028302D37293A200000282B293D506F16
:1023F000732B312020282D293D506F732D31202043
:10240000282A293D506F732B31302020285F293D29
:10241000506F732D313020202853293D536176654C
:1024200020506F73202028455343293D43616E633C
:10243000656C0D0A282E293D5472696D2B312028B8
:102440002C293D5472696D2D3120283A293D547252
:10245000696D2B313020283B293D5472696D2D3137
:1024600030202854293D53617665205472696D20CF
:102470002843293D436F6E6669670D0A2858293D38
:1024800053657420616C6C20706F736974696F6E32
:102490007320746F2063656E746572202020287825
:1024A000293D53657420616C6C207472696D7320D2
:1024B000746F2063656E746572200D0A2845293D8E
:1024C0005365742065766572797468696E672066F5
:1024D000726F6D20454550524F4D20202020284FCF
:1024E000293D53657420536572766F73204F6E2FAC
:1024F0004F66660D0A00456E7465722053657276EC
:102500006F20436F6E6669672042797465202800EA
:10251000456E74657220536572766F204F6E2F4F33
:102520006666204269744D61736B20280000293A69
:1025300020002020202020202020202020202020BB
:10254000202020202020202020202020202020208B
:102550002020202020202020200053656E64696EFA
:1025600067205353545620746573742070617474DB
:1025700065726E2E2028455343293D43616E636585
:102580006C0D0A0048656C6C6F00202020576F723C
:042590006C64000077
:10300000000EF86E200EF76E3A0EF66EF7EC0EF02C
:103010002CEC02F033EC02F082929EAA0DEF18F035
:1030200082823AEC02F0116E720E115CD8B42FEF6E
:1030300018F0730E115CD8B465EF18F06C0E115CCB
:10304000D8B467EF18F0640E115CD8B469EF18F0CB
:103050006D0E115CD8B46BEF18F008EF18F0D00EBD
:10306000586E4EEC0AF085EC0AF0200E27EC02F0C8
:10307000A3EC0AF0200E27EC02F0900E586ED0EC74
:1030800009F030500BEC0FF0200E27EC02F023502B
:103090000BEC0FF0200E27EC02F080EC0DF04E6AE6
:1030A000C4CF4DF0C3CF4CF04CEC04F0040EA9ECAF
:1030B00004F0200E27EC02F087EC0DF02B0ED8A4C4
:1030C0002D0E27EC02F008EF18F008EF18F008EFCB
:1030D00018F008EF18F02CEC02F02A0ECC6F2F0E2F
:1030E000CD6FCC510BEC0FF02CEC02F0CD510BEC72
:1030F0000FF02CEC02F0D00E586E4EEC0AF0A3EC60
:103100000AF02CEC02F000EE5EF0010E2B6E6F0E5A
:103110002D6EAA0EEE6E2D2E89EF18F02B2E89EF54
:1031200018F04EEC0AF0A3EC0AF02CEC02F000EEE2
:103130005EF0010E2B6E6F0E2D6E2B5014EC0FF007
:103140003A0E27EC02F02D5014EC0FF0200E27EC75
:1031500002F02E6AEE50E85014EC0FF0200E27EC2F
:1031600002F02E2A2EA8C4EF18F02CEC02F02B50FF
:1031700014EC0FF03A0E27EC02F02D5014EC0FF087
:10318000200E27EC02F02E6A2D2EAAEF18F02B2E1F
:0C319000AAEF18F02CEC02F008EF18F089
:020000040020DA
:08000000CAFE00BABE00004276
:020000040030CA
:04000000FFFEFEFE03
:02000600FEFFFB
:00000001FF
